:100000000C9463000C948B000C948B000C948B006C
:100010000C948B000C948B000C948B000C948C042F
:100020000C948B000C948B000C948B000C948B0024
:100030000C948B000C948B000C948B000C948B0014
:100040000C940E050C948B000C948B000C948B007C
:100050000C948B000C948B000C948B000C948B00F4
:100060000C948B000C948B000000000024002700EF
:100070002A000000000023002600290000000008DC
:10008000000201000003040700000000000000005F
:10009000010204081020408001020408102001021F
:1000A0000408102000000000250028002B00040494
:1000B0000404040404040202020202020303030310
:1000C00003030200DE0611241FBECFEFD8E0DEBF1F
:1000D000CDBF11E0A0E0B1E0EAE5F1E102C005909A
:1000E0000D92A235B107D9F721E0A2E5B1E001C038
:1000F0001D92A638B207E1F710E0C3E6D0E004C0D5
:100100002197FE010E94A508C236D107C9F70E94B7
:1001100058050C94AB080C940000AF92BF92CF929C
:10012000DF92EF92FF920F931F93CF93DF936C01B7
:100130007B018B01040F151FEB015E01AE18BF0898
:10014000C017D10759F06991D601ED91FC9101904A
:10015000F081E02DC6010995892B79F7C501DF9162
:10016000CF911F910F91FF90EF90DF90CF90BF90B4
:10017000AF900895833081F028F4813099F0823077
:10018000A9F008958730A9F08830C9F08430B1F41F
:10019000809180008F7D03C0809180008F77809355
:1001A0008000089584B58F7784BD089584B58F7DD0
:1001B000FBCF8091B0008F778093B000089580913D
:1001C000B0008F7DF9CF1F93CF93DF93282F30E0BE
:1001D000F901E458FF4F8491F901E057FF4FD491A2
:1001E000F901E255FF4FC491CC23A9F0162F8111DC
:1001F0000E94BA00EC2FF0E0EE0FFF1FEC55FF4F0E
:10020000A591B4918FB7F894EC91111108C0D095D5
:10021000DE23DC938FBFDF91CF911F910895DE2BFA
:10022000F8CFCF93DF9390E0FC01E057FF4F24918C
:1002300082559F4FFC0184918823D1F090E0880F74
:10024000991FFC01E859FF4FA591B491FC01EC55B1
:10025000FF4FC591D49161110EC09FB7F8948C9156
:10026000E22FE0958E238C932881E223E8839FBFC1
:10027000DF91CF9108958FB7F894EC91E22BEC9336
:100280008FBFF6CFCF92DF92EF92FF920F931F9323
:10029000CF938B0190910001891759F09F3F09F48A
:1002A0004AC0CF911F910F91FF90EF90DF90CF90B8
:1002B0000895E2ECF0E0C491C7FDF3CF61E00E9445
:1002C0001101C1114CC0980150E040E062E17AE7B1
:1002D00080E090E00E94630869017A0181E0C81A19
:1002E000D108E108F10885B5887F846085BD980153
:1002F000220F331FA4EFB1E00E94820828EE33E002
:1003000040E050E00E944108C13009F4BEC0C23054
:1003100009F4CDC0C111C5CFC7BC20936A01309389
:100320006B0140936C0150936D0180916E0082606F
:1003300080936E00B6CF80930001E2ECF0E0C491B0
:10034000CF3F09F4AECFC13009F440C010F1C23044
:1003500009F45EC0C7FDA5CF61E00E9411019801BC
:1003600050E040E0C23009F079C064E274EF80E010
:1003700090E00E94630869017A0181E0C81AD108FF
:10038000E108F1088091B100887F85608093B10019
:10039000AECF14BC15BC94B5926094BD95B5916078
:1003A00095BD282F30E0F901E255FF4FE491F0E0D0
:1003B000EE0FFF1FEC55FF4F45915491F901E057A7
:1003C000FF4FE491E0936101C0E078CF109280008C
:1003D000109281009091810098609093810090919B
:1003E0008100916090938100282F30E0F901E2555F
:1003F000FF4FE491F0E0EE0FFF1FEC55FF4F4591EA
:100400005491F901E057FF4FE491E093600156CF1A
:100410001092B0001092B1009091B0009260909351
:10042000B0009091B10091609093B100282F30E01E
:10043000F901E255FF4FE491F0E0EE0FFF1FEC559C
:10044000FF4F4591549150935F0140935E01F90134
:10045000E057FF4FE491E0935D0130CF60E072E13F
:100460008AE790E00E94630869017A0181E0C81A76
:10047000D108E108F108C13009F039CF809181003D
:10048000887F81608093810032CFD0928900C092B2
:100490008800209366013093670140936801509370
:1004A000690180916F00826080936F00FACEC092E4
:1004B000B300209362013093630140936401509331
:1004C000650180917000826080937000EACE8E306A
:1004D00008F08E508770806480937C0080917A0051
:1004E000806480937A0080917A0086FDFCCF8091B1
:1004F00078009091790008953FB7F8948091570162
:1005000090915801A0915901B0915A0126B5A89B2C
:1005100005C02F3F19F00196A11DB11D3FBFBA2F95
:10052000A92F982F8827BC01CD01620F711D811D55
:10053000911D42E0660F771F881F991F4A95D1F7DA
:1005400008958F929F92AF92BF92CF92DF92EF92D7
:10055000FF924B015C010E947C026B017C010E94B6
:100560007C026C197D098E099F09683E73408105E4
:100570009105A8F321E0821A9108A108B10888EE3C
:10058000C80E83E0D81EE11CF11C81149104A10463
:10059000B10429F7FF90EF90DF90CF90BF90AF901C
:1005A0009F908F900895089590E080E008958F9235
:1005B0009F92AF92BF920F931F93CF93DF93CDB7CC
:1005C000DEB7A1970FB6F894DEBF0FBECDBF19A25C
:1005D000423008F44AE08E010F5D1F4F842E912CAB
:1005E000B12CA12CA50194010E944108E62FB9016C
:1005F000CA01EA3044F5E05DD801EE938D01232B6A
:10060000242B252B79F790E080E0109769F0FD010D
:1006100001900020E9F73197AF014A1B5B0BBD0148
:100620008EE691E00E948D00A1960FB6F894DEBF91
:100630000FBECDBFDF91CF911F910F91BF90AF90B3
:100640009F908F900895E95CD7CFFC010190002026
:10065000E9F73197AF01481B590BBC018EE691E0D9
:100660000C948D00CF93DF93EC0160E08E810E94AB
:10067000E30061E08E810E94E30060E08E810E94D1
:10068000E3008BE891E00197F1F7DF91CF910895B6
:10069000CF92DF92EF92FF920F931F93CF93DF934E
:1006A0006C017C0187E0E80EF11CD0E0C0E0062F71
:1006B00010E0B8010C2E02C0759567950A94E2F718
:1006C0006170F70181917F010E94E3002196C4309F
:1006D000D10579F7C601DF91CF911F910F91FF905E
:1006E000EF90DF90CF900C943203CF92DF92EF9295
:1006F000FF920F931F93CF93DF93EC01F62E642F9D
:100700008C810E94E3008D818F3F19F060E00E9490
:10071000E3000F2D10E08F8584FF25C06E0187E078
:10072000C80ED11CF12CE12CB8010E2C02C075951D
:1007300067950A94E2F76170F60181916F010E945A
:10074000E300FFEFEF1AFF0A88E0E816F10461F713
:10075000CE01DF91CF911F910F91FF90EF90DF902D
:10076000CF900C943203B80184E0759567958A9513
:10077000E1F7CE010E9448036F2DCE01DF91CF91AA
:100780001F910F91FF90EF90DF90CF900C94480352
:1007900040E0682F8EE691E00C94750381E00E94A2
:1007A000C8038BE39FE10197F1F70895CF93DF939F
:1007B000823029F490917D01986090937D0180931F
:1007C00081011092820180E48093830180E1809313
:1007D000840180E58093850161E0809172010E942F
:1007E0001101809173018F3F19F061E00E941101A6
:1007F00061E0809174010E941101CEE6D1E09E017A
:100800002E56314080917D0184FD0BC084E090E044
:1008100021962817390744F461E08E810E94110166
:10082000EECF88E090E0F4CF8BE39DE00197F1F705
:1008300060E0809172010E94E30060E080917401A9
:100840000E94E300809173018F3F19F060E00E94E5
:10085000E30080917D0184FD34C063E08EE691E089
:100860000E944803CBE4D6E4CE010197F1F763E0A0
:100870008EE691E00E9448032197F1F763E08EE64F
:1008800091E00E94480383E592E00197F1F762E06E
:100890008EE691E00E94480380917D0180620E9473
:1008A000C80384E080937E018CE00E94C8030E940C
:1008B000CE0382E080937F0186E0DF91CF910C949C
:1008C000C80380620E94C8038BE496E40197F1F7A5
:1008D00080917D0180620E94C80383E592E00197C8
:1008E000F1F780917D0180620E94C803D5CF90917D
:1008F0008101691710F06FEF690FE62FF0E0E25900
:10090000FE4F9489890F80680C94C80341E00E94CF
:10091000750381E090E008951F920F920FB60F9239
:1009200011242F933F934F935F936F937F938F93F4
:100930009F93AF93BF93EF93FF9380916201909148
:100940006301A0916401B0916501892B8A2B8B2BE7
:10095000D1F190915D01E0915E01F0915F018081A4
:10096000892780838091620190916301A091640145
:10097000B0916501181619061A061B069CF48091A1
:10098000620190916301A0916401B09165010197AA
:10099000A109B1098093620190936301A09364015E
:1009A000B0936501FF91EF91BF91AF919F918F91AE
:1009B0007F916F915F914F913F912F910F900FBE5B
:1009C0000F901F90189580910001E2ECF0E0E49107
:1009D0009FEF90930001E13051F030F0E23069F088
:1009E00060E00E94E300DECF10926E00F9CF90919C
:1009F0006F009D7F90936F00F3CF909170009D7F6B
:100A00009093700091E09093B0009091B100987F26
:100A100094609093B1001092B300E2CF1F920F92B6
:100A20000FB60F9211242F933F938F939F93AF9301
:100A3000BF938091530190915401A0915501B091C1
:100A400056013091520123E0230F2D3758F50196BE
:100A5000A11DB11D20935201809353019093540125
:100A6000A0935501B0935601809157019091580180
:100A7000A0915901B0915A010196A11DB11D809319
:100A8000570190935801A0935901B0935A01BF9117
:100A9000AF919F918F913F912F910F900FBE0F902B
:100AA0001F90189526E8230F0296A11DB11DD2CFE5
:100AB000789484B5826084BD84B5816084BD85B539
:100AC000826085BD85B5816085BD80916E00816045
:100AD00080936E00109281008091810082608093EB
:100AE00081008091810081608093810080918000ED
:100AF0008160809380008091B10084608093B10018
:100B00008091B00081608093B00080917A00846011
:100B100080937A0080917A00826080937A0080913D
:100B20007A00816080937A0080917A008068809357
:100B30007A001092C10082E00E94D6030E94CE0388
:100B400061E08DE00E94110160E087E00E941101E8
:100B500061E089E00E94110181E10E946702BC010D
:100B6000990F880B990B0E94340720E030E040E891
:100B70005AE30E94980720E030E44CE955E40E94D3
:100B800098070E94FC06CB016AE070E00E942D08E5
:100B900070935C0160935B0160E080E00E947704E9
:100BA0008DE091E00E94250361E080E00E947704DF
:100BB00088E191E00E94250368EE73E080E090E018
:100BC0000E94A10293E8E92E90E0F92E27E9C22EB7
:100BD00020E0D22E35EBA32E30E0B32E00E010E063
:100BE0000E94CE038EE00E946702EC0160E080E08C
:100BF0000E94770484E291E00E94250360E085E092
:100C00000E94770440905B0150905C01052C000C21
:100C1000660877084AE0C301B20177FE0EC041E0E2
:100C20006DE28EE691E00E94750366277727CB017F
:100C300064197509860997094AE00E94D70260E0A5
:100C400087E00E9477048AE291E00E942503CD3B71
:100C500022E0D2070CF433C060E08BE00E947704FE
:100C60008DE291E00E94250361E08BE00E94770411
:100C700081E391E00E942503F7018491F6019490AD
:100C8000F5018490882009F44AC081110E94BA00BD
:100C9000E82DF0E0EE0FFF1FEE58FF4FA591B49145
:100CA0008C919822E1F161E08DE00E94E30061E027
:100CB00080E00E94770486E391E00E942503CE0144
:100CC0008C5291408139914008F06DC060E08BE01A
:100CD0000E94770487E491E00E94250361E08BE0A5
:100CE0000E94770481E391E00E94250360E08DE09B
:100CF0000E94E30061E080E00E9477048EE391E0CF
:100D00000E94250368EE73E080E090E00E94A1025B
:100D10000115110509F464CF0E94000061CF60E065
:100D20008DE00E94E30061E080E00E9477048EE3A2
:100D300091E00E94250366E071E089E00E94420193
:100D400064EF71E080E090E00E94A10266E271E051
:100D500089E00E94420164EF71E080E090E00E942F
:100D6000A1026AE471E089E00E94420164EF71E04F
:100D700080E090E00E94A1026DE571E089E00E94B0
:100D8000420164EF71E080E090E00E94A10268E817
:100D900071E089E00E94420164EF71E080E090E040
:100DA0000E94A1028CCFCC32D1400CF0ABCF60E0DE
:100DB0008BE00E9477048DE491E08ECFEEE6F1E0C7
:100DC0001382128285E091E0918380838CE084839A
:100DD0008FEF85838BE0868385E0878384E080873F
:100DE00083E0818782E082871386148615861686C3
:100DF000178681E00C94D6030E9403076894B11112
:100E00000C94920708950E94770788F09F5798F0F6
:100E1000B92F9927B751B0F0E1F0660F771F881FFF
:100E2000991F1AF0BA95C9F714C0B13091F00E9419
:100E30009107B1E008950C949107672F782F8827C8
:100E4000B85F39F0B93FCCF3869577956795B39540
:100E5000D9F73EF490958095709561957F4F8F4FAF
:100E60009F4F0895E89409C097FB3EF490958095B4
:100E7000709561957F4F8F4F9F4F9923A9F0F92F60
:100E800096E9BB279395F695879577956795B795DE
:100E9000F111F8CFFAF4BB0F11F460FF1BC06F5FC4
:100EA0007F4F8F4F9F4F16C0882311F096E911C0D6
:100EB000772321F09EE8872F762F05C0662371F0F7
:100EC00096E8862F70E060E02AF09A95660F771F0B
:100ED000881FDAF7880F9695879597F9089557FD3B
:100EE0009058440F551F59F05F3F71F04795880F98
:100EF00097FB991F61F09F3F79F08795089512162F
:100F000013061406551FF2CF4695F1DF08C01616DA
:100F100017061806991FF1CF86957105610508948B
:100F20000895E894BB2766277727CB0197F90895A2
:100F30000E94AB070C941C080E940E0838F00E9417
:100F4000150820F0952311F00C9405080C940B085B
:100F500011240C9492070E946F0770F3959FC1F3C0
:100F6000950F50E0551F629FF001729FBB27F00D57
:100F7000B11D639FAA27F00DB11DAA1F649F6627AC
:100F8000B00DA11D661F829F2227B00DA11D621FFB
:100F9000739FB00DA11D621F839FA00D611D221FB5
:100FA000749F3327A00D611D231F849F600D211D99
:100FB000822F762F6A2F11249F5750409AF0F1F01C
:100FC00088234AF0EE0FFF1FBB1F661F771F881F85
:100FD00091505040A9F79E3F510580F00C940508B0
:100FE0000C9492075F3FE4F3983ED4F3869577958F
:100FF0006795B795F795E7959F5FC1F7FE2B880F2B
:10100000911D9695879597F9089597F99F6780E8C0
:1010100070E060E008959FEF80EC089500240A944A
:101020001616170618060906089500240A941216C3
:101030001306140605060895092E0394000C11F4F6
:10104000882352F0BB0F40F4BF2B11F460FF04C0A3
:101050006F5F7F4F8F4F9F4F089597FB072E16F4BA
:10106000009407D077FD09D00E94910807FC05D0B5
:101070003EF4909581959F4F0895709561957F4FAF
:101080000895A1E21A2EAA1BBB1BFD010DC0AA1FC9
:10109000BB1FEE1FFF1FA217B307E407F50720F0E1
:1010A000A21BB30BE40BF50B661F771F881F991F5C
:1010B0001A9469F760957095809590959B01AC01A5
:1010C000BD01CF010895052E97FB1EF400940E94E8
:1010D0007A0857FD07D00E94410807FC03D04EF460
:1010E0000C947A0850954095309521953F4F4F4F7D
:1010F0005F4F089590958095709561957F4F8F4FC4
:101100009F4F0895A29FB001B39FC001A39F700D90
:10111000811D1124911DB29F700D811D1124911DFF
:101120000895AA1BBB1B51E107C0AA1FBB1FA6172E
:10113000B70710F0A61BB70B881F991F5A95A9F780
:1011400080959095BC01CD010895EE0FFF1F05908D
:0A115000F491E02D0994F894FFCF0C
:10115A00FF0000000086048D00D402D30250524FD3
:10116A004A45435420425900534D4152544B454D30
:10117A00424F200054454D503A002A4300445259E8
:10118A0000534F494C0050554D503A4F4E00505560
:10119A004D503A4F4646004D4F4953540057455417
:0211AA00000043
:00000001FF
